:100000000110050013000000601C0000FF0000004C
:10001000020C3A751AFF22FFFFFFFF0216087E0648
:10002000900074E06F6007EFF0E4900077F09000CC
:1000300074E07001FE900077E004F0C39E50037FEF
:1000400000229000777406F07F012202172EE4FB55
:10005000EB25E025E02474F8120232EB25E025E0E0
:10006000247CF812024B0BBB02E622021176BB0184
:100070000689828A83E0225002E722BBFE02E32245
:1000800089828A83E49322EF8DF0A4A8F0CF8CF0CC
:10009000A428CE8DF0A42EFE22BC000BBE0029EFBA
:1000A0008DF084FFADF022E4CCF875F008EF2FFF5F
:1000B000EE33FEEC33FCEE9DEC984005FCEE9DFE2D
:1000C0000FD5F0E9E4CEFD22EDF8F5F0EE8420D274
:1000D0001CFEADF075F008EF2FFFED33FD400798E3
:1000E0005006D5F0F222C398FD0FD5F0EA22E88F32
:1000F000F0A4CC8BF0A42CFCE98EF0A42CFC8AF0AC
:10010000EDA42CFCEA8EF0A4CDA8F08BF0A42DCCAD
:100110003825F0FDE98FF0A42CCD35F0FCEB8EF006
:10012000A4FEA9F0EB8FF0A4CFC5F02ECD39FEE4EC
:100130003CFCEAA42DCE35F0FDE43CFC2275F00831
:10014000758200EF2FFFEE33FECD33CDCC33CCC51F
:100150008233C5829BED9AEC99E58298400CF5823A
:10016000EE9BFEED9AFDEC99FC0FD5F0D6E4CEFBAC
:10017000E4CDFAE4CCF9A88222B800C1B90059BA9A
:10018000002DEC8BF084CFCECDFCE5F0CBF97818C8
:10019000EF2FFFEE33FEED33FDEC33FCEB33FB10C2
:1001A000D703994004EB99FB0FD8E5E4F9FA2278DC
:1001B00018EF2FFFEE33FEED33FDEC33FCC933C9EE
:1001C00010D7059BE99A4007EC9BFCE99AF90FD8F8
:1001D000E0E4C9FAE4CCFB2275F010EF2FFFEE3318
:1001E000FEED33FDCC33CCC833C810D7079BEC9A57
:1001F000E899400AED9BFDEC9AFCE899F80FD5F0E0
:10020000DAE4CDFBE4CCFAE4C8F922EB9FF5F0EA9E
:100210009E42F0E99D42F0E89C45F022E8600FEC38
:10022000C313FCED13FDEE13FEEF13FFD8F122E82C
:10023000600FEFC333FFEE33FEED33FDEC33FCD83C
:10024000F122E6FC08E6FD08E6FE08E6FF22E6FBF2
:1002500008E6F908E6FA08E6CBF822ECF608EDF62F
:1002600008EEF608EFF622ECF208EDF208EEF208DE
:10027000EFF222D083D082E493F608740193F6085B
:10028000740293F608740393F6740473D083D082D7
:10029000E493F208740193F208740293F208740371
:1002A00093F27404738A838982E473E4F530E53051
:1002B00025E025E0247CF8C000120232C007745209
:1002C0002530F8E6FFFBE4FAF9F8D0071200DED09B
:1002D0000012024BE53025E025E0247CF8C0001236
:1002E0000232780712020CD00012024BE53025E0F2
:1002F00025E0247CF8120232EC4D4E4F6076E5305A
:1003000025E025E0246CF8120232E53025E025E0F6
:10031000247CF812023EC31201FB50037F0322E546
:100320003025E025E0246CF812023EC000E53025BF
:10033000E025E0247CF8120232D000C3EF9BF534B4
:10034000EE9AF533ED99F532EC98F531E47FFF7EC6
:10035000FFFDFCAB34AA33A932A831C31201FB4024
:10036000037F0322E53025E02400F8E533F208E5B9
:1003700034F28015E530C39402500BE53025E024BB
:1003800008F8E4F208F27F03220530E530640260E9
:100390000302029EE4F530E53025E02404F8E2FE95
:1003A00008E2FFE53025E02400F8E2FC08E2FDD396
:1003B0009FEC9E401EE53025E02404F8E2FE08E2B2
:1003C000FFC3ED9FFFEC9EFEE48F388E37F536F5C8
:1003D000358009E4F538F537F536F535AF38AE3701
:1003E000AD36AC35780712021F8F388E378D368CBC
:1003F00035900074E070447F03FEFDFCAB38AA37F3
:10040000A936A8351200DEE53025E025E02414F8F1
:10041000E2FB08E2F908E2FA08E2CBF8EB2FFFEA88
:100420003EFEE93DFDE83CFC780212020CE5302579
:10043000E025E02414F81202578033E53025E0254A
:10044000E02414F8E2FC08E2FD08E2FE08E22538A8
:10045000FFEE3537FEED3536FDEC3535FC78011213
:10046000020CE53025E025E02414F8120257E530AF
:1004700025E025E02414F8E2FC08E2FD08E2FE088D
:10048000E2FF780712020CE53025E02408F8EEF2CE
:1004900008EFF20530E530640260030203877F074E
:1004A000228E328F33E4F535F536F537900087E04C
:1004B000F536A3E0F537E4F534E5187016900077CB
:1004C000E0B4060FD3900091E09400900090E09487
:1004D00000401EE53425E02448F8E4F208F2E53453
:1004E00025E025E0243CF812027C00000000020513
:1004F000A8E53425E02449F9E3700219E3701AE510
:100500003425E02400F8E2FE08E2FFE53425E0248B
:1005100044F8EEF208EFF28057E53425E02444F881
:10052000E2FE08E2FFE53425E02400F8E2FC08E200
:10053000FD121B3BD3EF9537EE95364033E534255E
:10054000E02400F8E2FE08E2FFE53425E02444F868
:10055000EEF208EFF2E53425E02448F8E4F208F280
:10056000E53425E025E0243CF812027C0000000080
:10057000E53425E02400F8E2FE08E2FFE53425E05A
:1005800025E0243CF8C000E2FB08E2F908E2FA08A2
:10059000E2CBF8E4FCFDEB2FFFEA3EFEED39FDEC8B
:1005A00038FCD000120257E53425E02448F808E270
:1005B0002401F218E23400F20534E534C394025009
:1005C000030204A9E4F534E53425E02449F9C3E342
:1005D000953319E39532400205350534E534B4020C
:1005E000E6E5356402600302068574FF900089F039
:1005F000A3F0E4A3F0A3F0F534E53425E02448F8B3
:10060000E2FE08E2FF4E7003020685E4FCFDC00432
:10061000A905AA06AB07E53425E025E0243CF8E26D
:10062000FC08E2FD08E2FE08E2FFD0001201698E3C
:10063000388F39D390008AE09539900089E0953859
:100640004007E538F0A3E539F0C390008CE0953918
:1006500090008BE095385007E538F0A3E539F0E5D8
:100660003425E02404F8E538F208E539F2E53425CC
:10067000E02448F8E4F208F2E53425E025E0243CE3
:10068000F812027C00000000C2080534E534640260
:1006900060030205E922E4F534F533E53325E0256E
:1006A000E0243CF812027C000000000533E533B47E
:1006B00002E91218B0E4F533E53325E025E0243CE7
:1006C000F8C000E2FC08E2FD08E2FE08E2FFE533C4
:1006D00025E025E02474F812023EEF2BFFEE3AFEEF
:1006E000ED39FDEC38FCD0001202570533E533B488
:1006F00002C60534E534C3940540B7E4F533AF349E
:10070000E4FCFDFEC004A905AA06AB07E53325E01D
:1007100025E0243CF8E2FC08E2FD08E2FE08E2FFE6
:10072000D0001201698F388E378D368C35AB38AAE0
:1007300037A936A835C00074522533F8E6FFE4FC2B
:10074000FDFED0001200DE8F388E378D368C357866
:100750000712020C8F388E378D368C35E47FB87EC9
:100760000BFDFCAB38AA37A936A835D31201FB40E4
:1007700030E5382448FFE53734F4FEE53634FFFD34
:10078000E53534FFFCE53325E025E0246CF8120262
:100790004BE53325E02400F8740BF20874B8F280BE
:1007A0001EE53325E025E0246CF81202630000000A
:1007B00000E53325E02400F8E537F208E538F2E5F6
:1007C0003325E025E0243CF812027C00000000E51F
:1007D0003325E02448F8E4F208F2E533C3940250EC
:1007E00033E53325E02400F8E2FE08E2FFE5332597
:1007F000E02404F8EEF208EFF2E53325E02408F8EF
:10080000E4F208F2E53325E025E02414F812027C36
:10081000000000000533E533640260030206EE22A7
:1008200074FFF537F538E4FFFE02089CE532C39407
:1008300009501CE53225E0242AF8E2FC08E2FDE537
:100840003225E02428F8ECF208EDF2053280DD785C
:1008500004E2FD08E2783ACDF208EDF2E4F532E583
:100860003225E02428F8E2FC08E2FDC39538EC9537
:100870003750048C378D38D3ED9FEC9E4004AE0486
:10088000AF050532E532B40AD6E538244BFDE43530
:1008900037FCD3EF9DEE9C4011D2097F04121992D0
:1008A000900092EEF0A3EFF08002C209E4F535F576
:1008B00036F532E53225E02408F8E2F53308E2F5B2
:1008C00034AE33FFE4FCFD7B64FAF9F81200DEC0BD
:1008D00006C007E53225E0244CF582E43400F583B8
:1008E000E0FEA3E0FFFBAA06E4F9F8D007D0061269
:1008F0000169E5186022C3EF941EEE94005019E5DB
:100900003225E02410F8E4F208F2E53225E0240C68
:10091000F8E4F208F202098BC3E5349536FFE533BB
:100920009535FEE4FCFD7B64FAF9F81200DEC006A2
:10093000C007E53225E0244CF582E43400F583E07D
:10094000FEA3E0FFFBAA06E4F9F8D007D0061201E7
:1009500069E53225E02410F8EEF208EFF2AE33AF8D
:1009600034E4FCFD7B64FAF9F81200DEC006C0072F
:10097000E53225E0244CF582E43400F583E0FEA363
:10098000E0FFFBAA06E4F9F8D007D006120169E5FA
:100990003225E0240CF8EEF208EFF20532E532647D
:1009A0000260030208A322E4FD300520ED25E024C7
:1009B00053F582E43418F583E493FE740193FFED5C
:1009C00025E02433F8A60608A6078041300420ED70
:1009D00025E02433F582E43418F583E493FE7401B2
:1009E00093FFED25E02433F8A60608A607801EED48
:1009F00025E02423F582E43418F583E493FE7401A2
:100A000093FFED25E02433F8A60608A6070DBD02E6
:100A100098E4FDED25E0241CF8E2FE08E2FFED2558
:100A2000E0240DF9D3E39F19E39E4016ED25E02461
:100A30000CF8E2FE08E2FFED25E0241CF8EEF208D7
:100A4000EFF2ED25E02433F8E6FE08E6FFEEC313EF
:100A5000FEEF13FFED25E0240DF9D3E39F19E39E8C
:100A60005034ED25E02433F8E6FE08E6FFED75F09E
:100A700008A4245CF8A60608A607ED25E02433F8B0
:100A8000E6FE08E625E0FFEE33F8ED25E0241CC87D
:100A9000F208EFF2803CED25E02443F582E43418BF
:100AA000F583E493FE740193FFED25E0240DF9D363
:100AB000E39F19E39E401BED25E0241CF9E3C313DB
:100AC000FE09E313FFED75F008A4245CF8A6060800
:100AD000A6070DED64026003020A03E4FDED75F064
:100AE00008A4245CF8E6FE08E6FFED25E02420F8E3
:100AF000EEF208EFF20DBD02E42285BA3953BA0FC7
:100B000043BA10E4F533E53325E025E02474F81208
:100B10000263000000000533E533B402E9753305D4
:100B200075ABFF121A56E4F534E53425E025E024D0
:100B300074F8C000120232C004C005C006C00774B9
:100B4000842534F8E675F003A42455F582E4341BBB
:100B5000F583E493FB740193FA740293F9120295FE
:100B6000A804A905AA06AB07D007D006D005D00473
:100B7000EF2BFFEE3AFEED39FDEC38FCD00012020F
:100B80004B0534E534C39402409FE4F5AB121A568A
:100B9000E4F534E53425E025E02474F8C0001202C1
:100BA00032C004C005C006C00774842534F8E67559
:100BB000F003A42455F582E4341BF583E493FB741D
:100BC0000193FA740293F9120295A804A905AA06E2
:100BD000AB07D007D006D005D004C3EF9BFFEE9A39
:100BE000FEED99FDEC98FCD00012024B0534E53483
:100BF000C39402409E1533E5336003020B10E4F505
:100C000034E4753810753727F536F535AF38AE371B
:100C1000AD36AC35780712021F8F388E378D368C83
:100C200035E53425E025E02474F812023E1201690E
:100C30008F388E378D368C3574522534F8A60705DB
:100C400034E534B402BB8539BA22439F04E453C669
:100C5000DFE5C600B5C6F375830075820775FD0D27
:100C6000E4E5FEF4FF75830075820675FD0DE4E58D
:100C7000FEB50704F59E8003759E0078100000D82D
:100C8000FC53C6E043C60843C680759607759703B4
:100C900075830075820475FD0D85FE8F7583007563
:100CA000820375FD0DE4E5FEF4FF75830075820295
:100CB00075FD0DE4E5FEB50704F595800375958394
:100CC00075BE0E5392FE9001007F007E02E4F0A3F9
:100CD000DFFCDEFA78007F00E4F208DFFC78FFE456
:100CE000F6D8FD75818F020D17020000020E74E424
:100CF00093A3F8E493A34003F68001F208DFF480A5
:100D000029E493A3F85407240CC8C333C4540F44F4
:100D100020C8834004F456800146F6DFE4800B01CE
:100D200002040810204080901673E47E019360BC9A
:100D3000A3FF543F30E509541FFEE493A360010E66
:100D4000CF54C025E060A840B8E493A3FAE493A38D
:100D5000F8E493A3C8C582C8CAC583CAF0A3C8C5AE
:100D600082C8CAC583CADFE9DEE780BE7533077D66
:100D70000774017E00A833088005C333CE33CED874
:100D8000F9FFACACECFBE4EF5B7003D533E3ED6053
:100D90001D74017E00A805088005C333CE33CED86C
:100DA000F9FFACAEECFBE4EF5B70031D80E0AF330A
:100DB0007401A807088002C333D8FCF5AC7401A8FD
:100DC00005088002C333D8FCFFF5AD8FAE53AACF20
:100DD00085BA3C53BA0F43BA10E4F537F536F5350A
:100DE000F534121A56E4F53374842533F8E675F0B9
:100DF00003A42455F582E4341BF583E49374019332
:100E0000FA740293F91202958F3B8E3A8D398C3821
:100E1000AB37AA36A935A834C31201FB500C853B69
:100E200037853A368539358538340533E533C3940B
:100E30000240B5AF37AE36AD35AC34780212020C95
:100E4000E5372FF537E5363EF536E5353DF535E541
:100E5000343CF534AF37AE36AD35FC781012020CA9
:100E60008FB3AF37AE36AD35AC34780812020C8F85
:100E7000B28537B143AA30853CBA75AC0375ADC0B5
:100E800075AEC022121B037D01E4FF1218EC7F0136
:100E9000121AA27F01121AE6121C4F121C42121AD9
:100EA0007C12152712195D1219C6D2AF753E01E5E5
:100EB0003E24FD601714602024FE602D1460311460
:100EC0007003020F5324076003020F561217D81243
:100ED0001305753E04020F56D2D8E53F70FC120090
:100EE0003E121B6D753E06807D12029B8F3E807602
:100EF000D390007DE0940090007CE09400400CA32F
:100F0000E024FFF090007CE034FFF0D3900091E00B
:100F10009400900090E09400400CA3E024FFF09037
:100F20000090E034FFF0D3900093E09400900092A2
:100F3000E094004016A3E024FFF0900092E034FF1C
:100F4000F0E07002A3E0700312159A900079E004BB
:100F5000F07006900078E004F012142E120F888FC3
:100F60003E8003753E0490008DE0B40124E4784B8C
:100F7000F6FF121C4FE4F0F51CF51D00051DE51DE4
:100F80007002051CB42CF4E51CB401EF7F01121CA7
:100F90004F121081020E9F22E4F5307531081208BD
:100FA0001012186C1213A3121A2B900075EFF01286
:100FB000000EEF605F7F01121992AD07AC06D3906F
:100FC000007DE0940090007CE094004010ECC4F8B8
:100FD00054F0C868FCEDC4540F48FD802E30081151
:100FE000EDAE047803CEC313CE13D8F9FDAC068062
:100FF0001AC37825E2941E18E29400500EECC4F84F
:1010000054F0C868FCEDC4540F48FDAF05AE04129F
:1010100004918003AF3122900074E06034E49000CA
:1010200080F0A3F090007FE004F0700690007EE076
:1010300004F07F05121992D390007FE09F90007E0C
:10104000E09E4014E4FF1216D2E4900076F07F0395
:1010500022E490007EF0A3F0900074E0FF90007610
:10106000E06F602A1216D2900074E0900076F0785B
:101070004CE654F060187F0C121992900090EEF03C
:10108000A3EFF0900090E0C313F0A3E013F0AF31B2
:101090002220CA030211757841E67003021175E43B
:1010A000784BF6F53074412530F8E6FF742625308C
:1010B000F8A60774412530F8E4F60530E530B40AA7
:1010C000E4784BE6700320CA12E4F530742625302C
:1010D000F8E4F60530E530B40AF222E52624E060B3
:1010E0001724B0601A24E0602124F060332490704B
:1010F00043E4FF121AA2803C7F01121AA28035E459
:10110000FF121B967851A607802A785C7603087632
:10111000E8786476030876E8784FE64420F6801491
:10112000785C760008762878647600087628784F10
:10113000E654DFF6E52654F064807049E52745283B
:101140006043E527FE7C00E42528FFEC3EFEC3EF6C
:10115000940AEE9400402EE526540FFDBD0F19E4CD
:10116000F530E53075F008A4245CF8A60608A6075B
:101170000530E530B402EB22ED75F008A4245CF8EC
:10118000A60608A60722C0E0C0F0C083C082C0D077
:1011900075D008C2CF30CD0302124930CB4720CCE6
:1011A000447840A6CEE6FFC39480403075F003EF4C
:1011B000A42404F582E5F03416F583E493FB74016E
:1011C00093FA7402938B238A24F5250525E525706F
:1011D00002052414F912005EF5CE80097840E62558
:1011E00022F8E6F5CE30CC297840E6C3948040154D
:1011F000AB230525E525AA247002052414F9120065
:101200005EF5CE8050784006E62522F8E6F5CE80E1
:101210004420CB41AFCE7840E6FE7028BF1002805C
:1012200034BF2002802FBF5008784FE64401F6807B
:1012300024BF6008784FE654FEF680197841A60F67
:1012400018068011EEC3940A50087840E62441F84D
:10125000A60F784006784B7601D0D0D082D083D0CC
:10126000F0D0E032E4FFFEEE75F008A4245CF8E66E
:10127000FC08E6FDEE25E02411F9C3E39D19E39C8B
:10128000400D7401A806088002C333D8FC42070E43
:10129000BE02D4807DEEC394025077EE75F008A4B0
:1012A000245CF8E6FC08E6FDEE25E02411F9C3E332
:1012B0009D19E39C401DEE25E02415F9C3E3940A33
:1012C00019E39400400D7401A806088002C333D8C6
:1012D000FC4207EE75F008A4246CF8E6FC08E6FD75
:1012E000EE25E02415F9C3E39D19E39C4021EE258A
:1012F000E02411F9C3E3940A19E394004011EE24A9
:1013000002FD7401A805088002C333D8FC42070E11
:1013100080838F1822E4F531F532121B20E490000F
:1013200074F0900076F0A3F090007EF0A3F0A3F0AC
:10133000A3F0900094F0A3F0900090F0A3F0F521BA
:10134000F530E53025E0244CF582E43400F583E007
:10135000FEA3E0FF900088E02FF0900087E03EF0D1
:101360000530E530B402DB900087E0FEA3E0FF7CAF
:10137000007D0A120089900087EEF0A3EFF0120DB5
:101380005C120AEA1206868019E530C3940A5012EC
:10139000E53025E02428F8740BF20874B8F2053023
:1013A00080E77F0A12199290007CEEF0A3EFF01212
:1013B0001B6D22E4F532E53225E02404F8E2FE0854
:1013C000E2FFE53225E02400F8E2FC08E2FDC39FDD
:1013D000EC9E5048E53225E02405F8C3E29DF53443
:1013E00018E29CF533FEAF34E4FCFD7B64FAF9F8B7
:1013F0001200DEC006C007E53225E0244CF582E489
:101400003400F583E0FEA3E0FFFBAA06E4F9F8D080
:1014100007D0061201698E358F368009E4F533F561
:1014200034F535F536D3E536940AE53594004002B7
:10143000D2080532E532640260030213A622E4F505
:1014400030E53075F008A4245EFFE53025E0240C7B
:10145000F8E2FC08E2FD121B82E53075F008A424D6
:1014600060FFE53025E02408F8E2FC08E2FD121BED
:1014700082E53075F008A42462FBC003E53025E066
:101480002400F8E2FE08E2FFE4FCFDE53025E0255B
:10149000E0246CF812023EEF2BFFEE3AFEED39FD30
:1014A000EC38FC780412020CAD07AC06D007121B16
:1014B000820530E530C394024087784FE6F520225C
:1014C0007DFF80707864E6FE08E6FFC37813E29F34
:1014D00018E29E40107874E6FE08E6FF7817E29F57
:1014E00018E29E504F780CE2FE08E2FF7809E22FE6
:1014F000F53418E23EF533780EE2FE08E2FF780B91
:10150000E22FFF18E23EAB07FAEB25E0FFEA33FEDD
:10151000C3E5349FE5339E50035305FAE53425E0D7
:10152000FFE53333FEC3EB9FEA9E50085305F58079
:10153000035305F08D1922E4F530784CF6FF121BA9
:10154000968F30E530BFFF06784D76058004784DE4
:1015500076FF784E7613E408F6785176FFFFEF2594
:10156000E02423F582E43418F583E493FC740193BA
:10157000FDEF75F008A4245CF8A60408A605EF7535
:10158000F008A4245EF8E4F608F6EF75F008A42449
:1015900060F8E4F608F6EF75F008A42462F8E4F6C3
:1015A00008F60FBF02B875224C22E4FBEB25E025BC
:1015B000E0247CF8120232EF2448FFEE34F4FEED12
:1015C00034FFFDEC34FFFCEB25E025E0246CF81241
:1015D000024BEB25E02400F8740BF20874B8F2EB30
:1015E000C394025017EB25E02408F8E4F208F2EB6C
:1015F00025E02404F8740BF20874B8F20BBB02ACBB
:1016000022EBC3940A5010EB25E02428F8740BF267
:101610000874B8F20B80EA22C0E0C0F0C083C08238
:10162000C0D075D000C000C004C005C006C007C24D
:101630008D758CD8758AF0051FE51F7002051EAEEA
:101640001EFF7C007D64120089ED4C7021900078B3
:10165000E0FEA3E0FFD3940AEE94004006A3EEF070
:10166000A3EFF0900078E4F0A3F0F51EF51FD0078B
:10167000D006D005D004D000D0D0D082D083D0F016
:10168000D0E03208840102FFFFFFFFFFFF048C005F
:10169000000000604A004C02D002B2006400640006
:1016A0006400640064006401020408050607080081
:1016B000000000000000000000000000000000002A
:1016C000000000000000000000000000000000001A
:1016D000000000000000000000000000000000000A
:1016E000000090008DE0705504F0E4FEFDFC7401F4
:1016F000A804088002C333D8FCF9FB900076E05BB5
:10170000B50313EC2404FA7401A802088002C33361
:10171000D8FC42068003E94206EF5BB50305E942C7
:10172000058011EC2404FB7401A803088002C33374
:10173000D8FC42050CBC02B6EE5D784CF622C0E047
:10174000C0F0C083C082C0D075D01053B9FD753DC4
:10175000007484253DF8E675F003A42455F582E471
:10176000341BF583E493740193FA740293F9120223
:1017700095E53D25E025E02474F812024B053DE592
:101780003DC3940240CB753F00D0D0D082D083D0EF
:10179000F0D0E032FE0000FE0008FE0004FE000C67
:1017A000FE0008FE0010FE000CFE0014FE0010FEFD
:1017B000001800007400007C00008400008C000011
:1017C00018010075010074010076FE0014FE001C73
:1017D00001007801009201008D0100900100640178
:1017E000006CFE0020FE0048E4FFFE74842EF8E644
:1017F0009018639342070EBE02F1EF42D4EF42F419
:10180000EF42E4EFF452DC75AA3B75BA0C43BA40E0
:1018100043B92053B9BF8FB4E4F5B375B24E75B177
:101820002075BBFF75A950F5AB75AC0375ADC075E0
:10183000AEC0220028002800320032003200320000
:101840003200320032003200320032003200320008
:10185000320032007800780032003200320032006C
:1018600032003203E803E800320032003200320076
:101870003200320102040810204080847810E2FE19
:1018800008E2FF8E32F5337D01ED25E02410F8E209
:10189000FA08E2FBC39533EA953250048A328B335F
:1018A000D3EB9FEA9E4004AE02AF030DBD02DA788F
:1018B00026E532F208E533F27824EEF208EFF22260
:1018C000121A56E4F53974842539F8E675F003A444
:1018D0002455F582E4341BF583E493740193FA7480
:1018E0000293F9120295E53925E025E02474F812F7
:1018F000024B0539E539C3940240CB22E4FE7C0259
:10190000ECC39402500E74842CF8E6901863934252
:10191000060C80ECEF6005EE42D48004EEF452D465
:10192000EEF4FF52F4EE42E4ED6005EE42EC80038B
:10193000EF52ECEF52DC22E4FFFEEE75F008A42437
:101940005DF8E624FBFD18E634FFFCEE25E0240DEF
:10195000F9C3E39D19E39C400D7401A806088002B9
:10196000C333D8FC42070EBE02D08F1B227E007FFD
:1019700064E4FDED25E024C6F582E4341AF583E441
:1019800093F4601DED25E024C7F582E4341AF58355
:10199000E493FCEF2DF582E43EF583ECF00DBD10F1
:1019A000D222753900753A647B017A00BFFF057F4A
:1019B000017E0022E53A2FF582E43539F583E07A9D
:1019C00000FB90007AE0FCA3E0FDAF037E00120074
:1019D00077AA06AB072243F80875CD4053CC7F4366
:1019E000CC4043CC2043CC1043CC0453CCFD43CB60
:1019F0000243CB0153CBBF43E80853E5FC43E3026A
:101A000043F50343900343ED0322A907E4FDFC746F
:101A1000017E00A804088005C333CE33CED8F9FF79
:101A2000E9FBE4EF5B600D7401A804088002C33396
:101A3000D8FC42050CBC02D7AF052212099712123E
:101A4000541214B0120003121927900074E0700DA4
:101A5000851832E5195232E51A52328003851B325D
:101A6000AF321219FA2275BF0F000000000000000B
:101A70000000000000000000000000D2D853B9FDB3
:101A800043B901E5B930E1FBE4F5BF22438901C266
:101A90008DD2A953B8FDE4F51EF51F900078F0A390
:101AA000F0A3F0A37464F0758CD8758AF0D28CD250
:101AB000AF22E4FE7D02EDC39402500E74842DF833
:101AC000E69018639342060D80ECEF6004EE4280CE
:101AD00022EEF452802200020101020103010402FD
:101AE000050606060702080A09020A020B280C016D
:101AF0000D030E01FF01EF600543D504800353D5AC
:101B0000FB53F5FB53E5FB43E30443ED04E4900092
:101B10008DF022E4F5E3439F10439F02FF0FBFFFC8
:101B2000FC539FEF75BE0EE4F5BFF5B975927622B2
:101B300053BAFEE5B920E004E53F6005E5B930E1C0
:101B4000FBE4F5BF53B9FE53B9FD22AB07AA06D398
:101B5000EB9DEA9C4007EB9DFFEA9CFE22C3ED9BB8
:101B6000FFEC9AFE22FF1BAAFF1BBDFF1BD0FF1B31
:101B7000E3FF1BF6FF1C09FF1C1CFF1C2F75BF0F8A
:101B800043B92053B9FD43BA01753F0143B901D2AE
:101B9000D822AB07AF04AE05C2AFA803A607E8047E
:101BA000F8A606D2AF22E4FFF582F5837420FEE4A6
:101BB00093F42FFFA3EEB583F62253B9EF788DA6E9
:101BC000B708A6B608A6B5788C1202322253B9EF30
:101BD000788DA6EB08A6EA08A6E9788C12023222D4
:101BE00053B9EF788DA6F308A6F208A6F1788C1207
:101BF00002322253B9EF788DA6FB08A6FA08A6F99F
:101C0000788C1202322243B910788DA6B708A6B696
:101C100008A6B5788C1202322243B910788DA6EB53
:101C200008A6EA08A6E9788C1202322243B9107895
:101C30008DA6F308A6F208A6F1788C120232224390
:101C4000B910788DA6FB08A6FA08A6F9788C1202BE
:101C50003222C2DA53D80F43D8D0D2D8D2D922EF09
:101C60006003D29222C29222FFFFFFFFFFFFFFFF1D
:00000001FF
